:020000040000FA
:100000000C2882073F3406345B344F3466346D3439
:100010007D3407347F346F3483160C3085008601BD
:100020008312803081008601A501A601A701073057
:100030009F00051D1F288519E428A901B428A60AD8
:100040004C2005199028851405105E3086004C2040
:10005000063086004C20393086004C2079308600EE
:100060004C208601851020280230A1000000A00B42
:100070003628A10B362800340A30A1000000A00B5E
:100080003E28A10B3E2800346430A1000000A00BE4
:100090004628A10B46280034FA30A1000000A00B2E
:1000A0004E28A10B4E2800340F30A2000000A00BF8
:1000B0005628A10B5628A20B56280034271D692864
:1000C000A71B7628A80F64302806031D0034A8015A
:1000D000A7172715A50A0A302506031D0034A50118
:1000E000A60A0A3026060319A6010034A80F053017
:1000F0002806031D0034A8016928A7190034A71594
:10010000A503FF302506031D00340930A500A60312
:10011000FF30260603198D280034A601A5010034FE
:10012000A50A051D99282508063A031D9028A50152
:1001300090280830A2009F20A20B9B28AD28051410
:100140000830860044204030860044200830860075
:100150004420013086004420003425080120860018
:100160004C20051DB02890280830A200BA20A20B10
:10017000B628C72885140830860044208510000062
:100180000514850008308600442005100034290835
:10019000A601A603A60AF63E0318CA280A3EA50031
:1001A00025080120860005143420051026080120AA
:1001B0008600851434208510A90A2908643A031999
:1001C000A9010519D028B428A508031DEC28A60804
:1001D000031DEC280517ED280513051D5E20851D60
:1001E0007D2005142508012086003C20051086018D
:1001F00085142608012086003C208510860185197B
:0E020000A711051DE4282711A713A801E42863
:02400E00503F21
:00000001FF
